:100000000AC018951895189518951895189518956B
:100010001895189518958FE181BD87E181BD8FED09
:100020008DBFC0ECE8EB4E2EDD275D2EEEE7F0E055
:10003000A0E6B0E088278D933197E9F780E489B98D
:1000400088E18AB948D16624E0E6F0E080E48FD107
:1000500058E0C895802D85D131965A95D1F704C0C6
:100060000E1111110E202020E0E8F0E088E47FD18D
:1000700058E0C895802D75D131965A95D1F704C0B6
:10008000040E1F2020202020E0EAF0E080E56FD160
:1000900058E0C895802D65D131965A95D1F704C0A6
:1000A00020202020201F0E04E0ECF0E088E55FD146
:1000B00058E0C895802D55D131965A95D1F704C096
:1000C0002020201F1F202020ECD08CE050D167C0C2
:1000D000F9D110E90DD211EA0BD219E109D201D2FE
:1000E000F1D110E905D212EA03D214E101D2F9D11B
:1000F000E9D110E9FDD111EAFBD1F3D1E3D111E946
:10010000F7D111D2A2E61C93ECD1DCD110E9F0D1E9
:1001100012EAEED1E6D1D6D111E9EAD104D2A3E6B2
:100120001C93DFD1CFD110E9E3D11CEAE1D1D9D1C1
:10013000C9D111E9DDD1F7D1A4E61C93D2D12FC0EA
:10014000C1D110E9D5D118EAD3D1CBD1BBD111E9B6
:10015000CFD1E9D1A5E61C93C4D10895B3D110E95C
:10016000C7D119EAC5D1BDD1ADD111E9C1D1DBD11A
:10017000A6E61C93B6D10895A5D110E9B9D11CEA21
:10018000B7D1AFD19FD111E9B3D1CDD1A4E61C93A2
:10019000A8D198D110E9ACD110E0AAD1A2D192D1C6
:1001A00010E9A6D111E0A4D19CD18CD110E9A0D145
:1001B00018E19ED196D186D110E99AD110E098D15C
:1001C00090D180D111E994D1B0D1A0E61C93ABD1EC
:1001D000A1E61C9386D1E1E0F0E074D000916100CB
:1001E000003809F004C085E08093610003C080E01E
:1001F000809361008FE711E063D0E0E6F5E04BD03B
:100200008FEB11E05DD0E2E7F5E045D0A8EAB0E081
:10021000E0E6F0E008D137D0E8E7F5E03CD0A8EA26
:10022000B0E0E1E6F0E0FFD02ED080E09AD0EAE73F
:10023000F5E031D0ECE7F5E02ED0A8EAB0E0E0E65A
:10024000F0E0F1D00BD0E8E7F5E010D0A8EAB0E09C
:10025000E1E6F0E0E8D002D00FD0A1CFA8EAB0E00C
:100260008D91882311F00BD0FBCF0895BBD0802D4A
:1002700011F005D0FBCF08958DE001D08AE05D9BA1
:10028000FECF8CB90895A8EAB0E08D91882311F0D3
:1002900068D0FBCF0895A6D0802D11F062D0FBCF9F
:1002A000089581E064D014D080E861C08FE72130E8
:1002B00039F08FEB223021F08FE8233009F08FECFA
:1002C000810F55C088EE93E07ED03197D9F708951D
:1002D00083E0992778C08AEF90E075D0B89AB99AF0
:1002E000BA9ABB9ABE9ABF9AC798EF93FF93E6EF6C
:1002F000F0E05DD0FF91EF91C698C098C198C29A86
:10030000C39AC69AEF93FF93E6EFF0E050D0FF91C7
:10031000EF91C69855D0C69AEF93FF93E6EFF0E0C1
:1003200046D0FF91EF91C6984BD0C69AEF93FF93BA
:10033000E6EFF0E03CD0FF91EF91C69841D0C39832
:10034000C69AEF93FF93E6EFF0E031D0FF91EF9183
:10035000C69836D088E20BD08EE009D086E007D070
:100360000895C79A829505D004D02AD00895C798D9
:10037000F9CF859510F4C39A01C0C398859510F400
:10038000C29A01C0C298859510F4C19A01C0C19863
:10039000859510F4C09A01C0C098C69AEF93FF9358
:1003A000E6EFF0E004D0FF91EF91C6980895319701
:1003B000F1F70895689462F80895E89462F8089552
:1003C00081E090E000C0EF93FF93EE27E82BE92B4C
:1003D00031F0E4ECF9E03197F1F70197D1F7FF91B3
:1003E000EF910895C895319600200895000F111FD0
:1003F000221F331F089500951095209530950F5FAB
:100400001F4F2F4F3F4F0895019110810EC0019152
:100410001191219130810BC00191108117FF05C00E
:100420003FEF2FEF04C0008111272227332737FF2A
:1004300003C0E1DF8DE28D93CF93DF93CF92DF9204
:10044000EF92AA24BB24CC24DD24EE2440E2CAE0AF
:10045000DD2755E093E38881890F87FD9F7083FD39
:10046000907F891B89935A95A9F7C0DFAA1CBB1CF2
:10047000CC1CDD1CEE1C4A9551F7E894EFE0FF27F9
:1004800082910ED0EB30E0F71EF068948A2D0CD0EC
:1004900088278D93EF90DF90CF90DF91CF910895D3
:1004A000982F829501D0892F8F70805D26F0803340
:1004B00009F4089568948D930895939892988B9871
:1004C0008A9808958A9A8B9804D08A9802D08B9A39
:1004D00000C0EF93FF93E9E0F0E069DFFF91EF9157
:1004E00008958A9A8B9AF5DF8A98F3DF8B98F1CF7B
:1004F0000894111F01C0110F59F08A9A18F40000D6
:100500008B9802C08B9A00C0E4DF8A98E2DFF3CFB9
:100510008A9A8B98DEDF8A98829BFECFE894839933
:10052000689462F8D6CF089401C08894331F11E014
:100530008A9A8B98CEDF8A98829BFECFCADF8894F6
:1005400083990894111FA0F78A9A379510F48B9815
:1005500001C08B9ABEDF8A98829BFECFBADF0895D6
:1005600054434E373520546865726D6F6D65746500
:1005700072002A2A2A2A20002C004300202A2A2A34
:020580002A004F
:00000001FF
